:020000040000FA
:0600000007309F00E0291B
:08000800BC00030EBD008B1AC1
:100010002B280B1A1B283D0E8300BC0E3C0E09003A
:10002000810183166400883081008312851490302A
:100030008B00BB0108008B100C30B700B70B1E28DB
:1000400006180B28AD30810020308B000230BB0039
:100050000830B7000B280B113B193E28B7080319CD
:100060003728060CB80CB703AD3081000B28061CEE
:1000700058280130BB003808B9005828BB19582847
:10008000B70803195028BA0C031C4928000085142E
:100090004C28851000000000B703B53081000B2804
:1000A0000000000000008514BB15A83081000B285B
:1000B00010308B000130BB050B2885100630BB00CB
:1000C0000000B5308100A0308B000830B700080078
:1000D00062213B1C68283B1008005D206221BB1890
:1000E0006E28080082071A2A292A292A202A292A62
:1000F000222ABF09C009C109C209BF0A031D8728F6
:10010000C00A031D8728C10A031D8728C20A2308C5
:100110004207A300220841070318A020A2002108DB
:10012000400703189D20A10020083F0703189A20CC
:10013000A0000800A10A031D0800A20A031D080070
:10014000A30A08003030BE02031908008720BE0B46
:10015000A62808004308BE003B30C2009A30C10008
:10016000CA30C0000030BF00A2204408BE000530E5
:10017000C200F530C100E130C0000030BF00A22055
:100180004508BE00C2019830C1009630C0008030E2
:10019000BF00A2204608BE000F30C1004230C000A0
:1001A0004030BF00A2204708BE000130C1008630A9
:1001B000C000A030BF00A2204808BE00C101273007
:1001C000C0001030BF00A2204908BE000330C000AC
:1001D000E830BF00A2204A08BE00C0016430BF0062
:1001E000A2204B08BE000A30BF00A2204C08BE006F
:1001F0000130BF00A2200800303080007920A31B0E
:100200000429800A8720FF287920080043308400D1
:100210003B30C2009A30C100CA30C0000030BF007D
:10022000FC20840A0530C200F530C100E130C00076
:100230000030BF00FC20840AC2019830C100963013
:10024000C0008030BF00FC20840AC2010F30C10012
:100250004230C0004030BF00FC20840AC20101309F
:10026000C1008630C000A030BF00FC20840AC2015B
:10027000C1012730C0001030BF00FC20840AC20139
:10028000C1010330C000E830BF00FC20840AC20175
:10029000C101C0016430BF00FC20840AC201C10159
:1002A000C0010A30BF00FC20840AC201C101C001A4
:1002B0000130BF00FC200800A001A101A201A301A0
:1002C000AA20080008003B1C63293B103908BA002B
:1002D0006D2039080800A401A501A601A701A80105
:1002E0002030A9002C08B0002D08B1002E08B20063
:1002F0002F08B3000310301C94292008A507031C05
:100300008629A60F8629A70F8629A80A2108A607ED
:10031000031C8D29A70F8D29A80A2208A707031CF3
:100320009229A80A2308A807A80CA70CA60CA50CBC
:10033000A40CB30CB20CB10CB00CA90B7A2901308F
:10034000A8000800243084000008AB000830AA0090
:10035000AB0C031CAF29861506150611B2298611B0
:1003600006150611AA0BA829840A29300402031CC9
:10037000A429861786130800C821C821C821C821CE
:10038000C821C8210800C821C821C821C8210800E7
:10039000CB21CB210800FF30B400D9298030B40034
:1003A000D9294030B400D9292030B400D9291030DF
:1003B000B400FF30B500B50BDB29B40BD929080018
:1003C0008B0183168113F53085000130860083127E
:1003D0000030A4000030A5000030A6000030A700C7
:1003E0000030A800A2211730AF00DC30AE0065302D
:1003F000AD00DE30AC00203036226B21A221A221DC
:10040000CB2110206820FE303902031D022A68200B
:10041000FE303902031D022A68205C303902031DB8
:10042000022A6820E0303902031D022A68203908B8
:100430007220022A3A225C216B21A221312208007B
:10044000602208003A225C216B21A22131228922FC
:10045000080008000D30BA006D200A30BA006D2087
:100460000800203084000030BE22080084000030E4
:10047000AF2208000A30B600433084008001840AAD
:10048000B60B3E2A0A30B6004C3084006820FD309E
:10049000390203195F2A3908CD000F39303EB608FA
:1004A0000319462A80008403B6034D0E0F39303EEF
:1004B000B6080319462A80008403B603462A0800BA
:1004C000203036220621FE30BA006D20FE30BA0000
:1004D0006D20E030BA006D205C30BA006D20033032
:1004E000BA006D200530B6004C3084000008BA0018
:1004F0003030BA02BA0E84030008BA073030BA02AC
:10050000BA0E6D208403B60B762AFD30BA006D203A
:100510000800FE30BA006D20FE30BA006D20E030D9
:10052000BA006D205C30BA006D20FB30BA006D203F
:10053000FD30BA006D200800FE30BA006D20FE309C
:10054000BA006D20E030BA006D205C30BA006D203A
:10055000FA30BA006D20FD30BA006D200800831615
:100560009B0083120430B60083161C141A089B0AE1
:100570008000840A8312B60BB42A080083169B00FD
:1005800083120430B6008B13831600089A009C0176
:100590001C1555309D00AA309D009C149C18CE2A35
:1005A0009C139B0A83128C13840AB60BC42A8B17E4
:0205B000080041
:02400E00093F68
:1042000028000100D600000080009F00D5000000BB
:10421000B000F600DA0000006400000000000000BA
:00000001FF
